:100000000C9446000C9463000C9463000C94630001
:100010000C9463000C9463000C9463000C946300D4
:100020000C9463000C9463000C9463000C946300C4
:100030000C9463000C9463000C9463000C946300B4
:100040000C9463000C9463000C9463000C946300A4
:100050000C9463000C9463000C9463000C94630094
:100060000C9463000C9463000C9463000C94630084
:100070000C9463000C9463000C9463000C94630074
:100080000C9463000C9463000C94630011241FBE55
:10009000CFEFD0E1DEBFCDBF11E0A0E0B1E0ECEDED
:1000A000F0E000E00BBF02C007900D92A030B10756
:1000B000D9F711E0A0E0B1E001C01D92A030B10776
:1000C000E1F70C9465000C940000CFEFD0E1DEBFA7
:0C00D000CDBF81E090E00C946D00FFCFEC
:00000001FF
